S123E0000E8E1FFF7F1C9F7F1CA27F1C027F1D777F1C007F1C017F1CA37F1D5C7F1D5D862F
S123E02009B71D5FCE0800FF1C23FF1C25FF1C218604CE1D6F6F00084A26FA8604CE1D7363
S123E0406F00084A26FA8606CE1D7A6F00084A26FA7C1D7ECE1CA6FF1CA06F006F01EF02D7
S123E060EF046F066F086F0C6F0E6F0F731C9F8608B71C15861FC6FFCE1D3EA700E7016F12
S123E08002080808C04082007A1C1526EECE1D3E86FFA70201B640007F1C038603B7C0082D
S123E0A08612B7C008B6C009CEC010A60184FBA70186FFA7008635A701A6018A08A7018466
S123E0C0F7A70186B8A700A60384FBA7036F00A7028636A703CEC0188604A7028608A70357
S123E0E06F046F058601A7068636A70786A1A7018690A70086A0A7018690A700CEC000866C
S123E100C3A7054FA7048668A70386CCA707B71D58A6007EE6AC3637CEF926BDF37DFE1C77
S123E120A0FF1C17FF1C19C608A600BDF2B9BDEBD1BDEBD1A601BDF2B9BDEBD18620BDF22A
S123E1404EBDF24EA606BDF2B9A607BDF2B9BDEBD1EE06A606BDF2B9A607BDF2B9BDF2976B
S123E160FE1C195A270AEE04FF1C19BC1C1726B9BDF2973332397D1CA326FB3637FF1C110F
S123E180FE1CA0E600260153F71CA3CE1D2686086F006F0108084A26F7CE1D26FF1C15FE77
S123E1A01CA0FF1C13C608FE1C13EE04BC1CA02721FE1C15B61C13A700B61C14A70108086B
S123E1C0FF1C15FE1C13EE04FF1C135A26D90D7EE2B2FE1C15B61C13A700B61C14A701C637
S123E1E008CE1CA6FF1C1337C608CE1D26FF1C15FE1C15EE00BC1C1326037EE292FE1C15BD
S123E2000808FF1C155A26E833BDE36825C0FF1C15B61C11F61C12FE1C15E70009A700092C
S123E2206F00096F00096F00096F000907A70009FF1C11FE1C13B61C11F61C12A706E70748
S123E2406F086F096F0C6F0D6F0E6F0FB61CA0F61CA1A704E705FE1CA0A602E603FE1C13A5
S123E260A702E703FE1CA0B61C13F61C14A702E703FE1C13EE02B61C13F61C14A704E705F0
S123E280FE1CA0E600BDE384FE1C13A700E7010C2020B61C14F61C138B10C900F71C13B762
S123E2A01C14FE1C150808FF1C15335A27037EE1E70D077F1CA3063332397D1CA326FB4D1E
S123E2C026040C7EE3143637FF1C11FE1CA0E6001127075D260153F71CA3FE1CA0C608A161
S123E2E000270CEE04BC1CA027275A26F220228D2E8D5BFE1CA0C608A10126088D2136A6F6
S123E300008D4B32EE04BC1CA027095A26EA0C20030D2000077F1CA306FE1C113332393645
S123E32037FF1C11EE02FF1C13FE1C11EE04FF1C15B61C13F61C14A702E703FE1C13B61C6E
S123E34015F61C16A704E705FE1C113332393637CE1D3EC608A10227090808085A26F60D4A
S123E36020036F020C333239368608CE1D3E6D0227090808084A26F60D20078D07A702EEF2
S123E380000C323937FF1CA4B61CA24D26067C1CA2B61CA2CE1D3EC608A10227F1080808A7
S123E3A05A26F6FE1CA433393637FF1D78B61D78F61D79FE1CA0A70EE70F3E333239B6C02A
S123E3C0088580270884DFB7C008B6C00901B6C00685802705B6C0018580B6C01385C0277D
S123E3E003B6C012B6C01185802714B6C0107D1C9F2716B61D5B8478BDF50D4FBDF411B61C
S123E400C01185402703B6C0103BCE1D7AA6008B0119262AC602A70008A6008B01198160D4
S123E420261C4F5A26F06F0008A6008B01198124260C6F0008A6004C810826028601A700F6
S123E440C604CE1D72A6008B01A7002604095A26F4B61D72851F261CF61D58CA407D1C02D6
S123E4602609C4BF86FFB71C0220037F1C02F71D58F7C0077D1C9F273D4F36FE1CA0A60E13
S123E480AA0F270FA60EE60F5A26044D27014AA70EE70F324C36EE04BC1CA026E13386080C
S123E4A0FE1CA0AF06EE04FF1CA0AE06C1012706A60EAA0F26EA3B3434C60530A602A7002F
S123E4C0085A26F830C6E486FDE705A706A601B1E4FC230AC6E58655E705A706201D5F485A
S123E4E059AB06E905A706E705EE05EE00FF1D5930B61D59F61D5AA705E7063B2AF24EF238
S123E5005EF26AF277F329F282F2B9F2A9F37DF297F405E176E2BAF409ED1EE116F3B6F37E
S123E520D3F3E5F3F7F398F3A3F2D6F411F426F43BF458F475F4A7F50DF546F589F59AF57C
S123E540AEF5CEF5D2F648F64CF650F652E3A8F200E555E55537CEF9AEBDF37DBDEBD186A8
S123E56028BDF24E32BDF2B98629BDF24EBDEBD18670BDF24E8663BDF24EBDEBE030EE0034
S123E580BDF2A9BDEBD18650BDF24E8649BDF24E8644BDF24EBDEBE0BDF409BDF2B9BDF2E7
S123E5A09739BDF297CEF9E4BDF37DBDF43BBDF2008656BDF24ECEFA2CBDF37DBDF4A7BDBF
S123E5C0F2008656BDF24ECEF9FABDF37DBDF458BDF2008643BDF24ECEFA15BDF37DBDF445
S123E5E075BDF2008643BDF24EBDF297BDF59A37CEE61F4D2703CEE651BDF37D4F33CE1D7B
S123E60065BDF1BBCE1D65BDF22DBDF64C8101270481022606CEE67BBDF37DBDF297390DB9
S123E6200A526164696F2063757272656E746C7920706F7765726564206F666620616E6411
S123E6402073657420746F206368616E6E656C20000D0A526164696F20697320706F776551
S123E660726564206F6E20616E642073657420746F206368616E6E656C20000D0A0A412001
S123E68070726F6365737320686173207369676E616C6564206120706F77657220646F777C
S123E6A06E2070726F63656475726500BDF2A2B6C010B6C012B6C0118A80B7C0117F1C1FCD
S123E6C0CEF7A5BDF37DBDE5A2BDF297CEF8D2BDF37DCEF654BDE1762517CEF8E9BDF37D0C
S123E6E0CEF6B7BDE1762509CEF9C9BDF37DBDF297860DBDF24E4FF61C1FCE1D65BDF1BB8D
S123E700CE1D65BDF22D863EBDF24EBDF2D67D1C3627DECE1C36FF1C34A6008120260608C5
S123E720FF1C3420F481032740810D27C4810A27C081202DBC7C1C1FBDF297BDF297FF1CB4
S123E7400DCEFA57BDE76A4D2608CEF803BDF37D209FFE1C0DFF1C34CEFA984A27040808F0
S123E76020F9EE00AD007EE6F102FF1C0FFF1C11FE1C0DFF1C1386018D252522FE1C116DC7
S123E7800027030820F9086D0026034F2010FF1C11FF1C0FFE1C13FF1C0D4C28DB4F393655
S123E7A037FE1C0DA600271208FF1C0DFE1C0FE600270708FF1C0F1127E74D27118120270D
S123E7C00D810D2709810A270586FF0C20145D270FC120270BC10D2707C10A27030C200229
S123E7E04F0D333239CEFABABDF37D393637CE0000FF1C1BCE1BFFFF1C1DFE1C34A6002787
S123E80010BDF329FF1C1B81202606BDF329FF1C1DCEE835BDF37DBDF25E81792611FE1C87
S123E8201B6F0008BC1C1D26F8CEE84CBDF37DBDF2973332390D0A41726520796F752073DD
S123E8407572652028792F6E293F20000D0A4D656D6F727920636C65617265642E00363767
S123E860FE1C25FF1C1BFF1C1D7C1C1DFE1C34A6002726BDF329FF1C1BF61C1CC4F0F71CED
S123E8801CFF1C1D7C1C1D8120260EBDF329FF1C1DB61C1E84F0B71C1EBDF297CE1C86FF7B
S123E8A01C15FE1C1BBDF2A98609BDF24EC610A60008FF1C1BBDF2B9FE1C1581202C028664
S123E8C02E817F2602862E847FA70008FF1C158620BDF24EFE1C1B5A26D5CE1C868620BD48
S123E8E0F24EBDF24EBDF24EC610A600BDF24E085A26F7BDF297B61C1BB11C1D269EB61C2F
S123E9001CB11C1E2396FE1C1BFF1C25BDF2973332393637FE1C23FF1C1BFE1C34A60027DF
S123E92006BDF329FF1C1BBDF297FE1C1BBDF2A98620BDF24EBDF24EA600BDF2B9862DBDCD
S123E940F24E8620BDF24EBDF2D6FE1C34EE008C0D002609FE1C1B08FF1C1B20CAFE1C349C
S123E960A6008120260608FF1C3420F14D27B8812B2720812D272D812E2736810D2714BD05
S123E980F329FF1C15B61C16FE1C1BA70008FF1C1B20CA08FF1C346D002707FE1C1B08FF0D
S123E9A01C1B20B908FF1C34FE1C1B09FF1C1B20ACBDF297FE1C1BFF1C233332393637BD2B
S123E9C0E1163232393637FE1C34A6002608CEF832BDF37D200EBDF329BDE1762406CEF9DF
S123E9E046BDF37DBDF2973332393637FE1C34A6002608CEF982BDF37D2014BDF329FF1C8F
S123EA0011B61C12BDE2BA2406CEF96DBDF37DBDF29733323936378614B71C27FE1C21FFFA
S123EA201C1BFF1C1D7C1C1DFE1C34A600271CBDF329FF1C1BFF1C1D7C1C1D8120260CBDEB
S123EA40F329FF1C1D4F9800B71C27FE1C1BBDED1EFF1C28FE1C1BBDF2A98609BDF24EFE26
S123EA601C1B5F8620BDF24EA600BDF2B9085CBC1C2826EF8609C1032703BDF24EBDF24E5B
S123EA80CE1C36BDF37DBDF297FE1C28FF1C1B7D1C272B057A1C272710B61C1BB11C1D2686
S123EAA0AAB61C1CB11C1E23A2FE1C1BFF1C213332393637FE1C23FF1C1BFE1C34A6002601
S123EAC008CEF832BDF37D2020BDF329FF1C9DAD003607B71C9632B71C97F71C98FF1C99E6
S123EAE0BF1C9BCEF84ABDF37D3332393637CEF869BDF37DB61C96BDF2B9BDEBD1F61C9607
S123EB00CEFA468608B71C1159240AA6002712BDF24E0820F6A6002708088620BDF24E2050
S123EB20F48620BDF24E087A1C1126DCBDF2978641BDF24EBDEBE0B61C97BDF2B9BDEBD1AD
S123EB408642BDF24EBDEBE0B61C98BDF2B9BDEBD18658BDF24EBDEBE0FE1C99BDF2A9BDEE
S123EB60EBD18653BDF24EBDEBE0FE1C9BBDF2A9BDEBD18650BDF24E8643BDF24E8D61FE6C
S123EB801C9DBDF2A98D4ABDF297BDF297FE1C9DBDED1EFF1C28FE1C9DBDF2A98609BDF2EE
S123EBA04EFE1C9D5F8620BDF24EA600BDF2B9085CBC1C2826EF8609C1032703BDF24EBD8C
S123EBC0F24ECE1C36BDF37DBDF297BDF2973233393637C6048620BDF24E5A26FA33323988
S123EBE0368620BDF24E863DBDF24E8620BDF24E323936377F1C9FCEFFFFFF1C1B08FF1C9E
S123EC001DBDF25E810D27F9810A27F58153270A81732706813A274520E7BDF25E8139272F
S123EC203A81382736813727328131270881322704813326CCC60136BDECB2B71C111B169D
S123EC40328D36802EB71C12B61C11B01C12B71C118D528D5D1B1627A8207520795FBDEC84
S123EC60B24D2772B71C111B1686318D0C8D438D348D3F1B16278A205736CE1C13802FB744
S123EC801C12A601A7008D2AA7011B167A1C1226F1EE00BC1C1B2203FF1C1BBC1C1D23034E
S123ECA0FF1C1D32398D0BA700081B167A1C1126F43937BDF25E8D0D1658585858BDF25EDA
S123ECC08D031B3339803081112D028007840F39CEF872BDF37DCEF88EBDF37DFE1C1BBD7D
S123ECE0F2A9CEF8B0BDF37DFE1C1DBDF2A9BDF297731C9F3332393637CEF815BDF37D3389
S121ED00323936378601BDF3B633323936374FBDF3B633323936374FBDF411333239B2
S123ED1E3637FF1C2CCE1C36FF1C2A6F00FE1C2CE60008FF1C2CCEEEECA60008E100260968
S123ED3ECEEEDDBDEE2C7EEDE8084A26EF1784C0264017843FCEEF29BDEE48C1202D04C140
S123ED5E302D037EEDE8FE1C2CA60008FF1C2C5F4D2A02C6FFFF1C2EBB1C2FF91C2EB71CA1
S123ED7E2FF71C2EFE1C2E8609BDEE1CBDEDF27EEDE881402627CEEFF117840FBDEE481704
S123ED9EC5202706BDEE5B7EEDE88609BDEE1C8600C41027028600BDEE1C7EEDE8C18D26F9
S123EDBE09CEEED9BDEE2C7EED648180260FCEF02517840FBDEE48BDEE5B7EEDE817CEF009
S123EDDE6D17840FBDEE48BDEE5B4FBDEE1CFE1C2C333239368624BDEE1CFF1C30B61C3013
S123EDFE8D07B61C318D023239363644444444BDF2CABDEE1C32BDF2CABDEE1C3239FF1CAC
S123EE1E32FE1C2AA70008FF1C2AFE1C323936FF1C2EA600271208FF1C2EFE1C2AA700083F
S123EE3EFF1C2AFE1C2E20EA323936374D2709E600085D26FA4A20F48DD433323936378609
S123EE5E09BDEE1C178430262B8623BDEE1CFE1C2C17840F810C2C0CA60008FF1C2CBDEEDF
S123EE7E077EEED6EE00BDEDF2FE1C2C0808FF1C2C7EEED6811026134FBDEE07FE1C2CA607
S123EE9E0008FF1C2CBDEE077EEED681202619FE1C2CA60008FF1C2CBDEE07862CBDEE1CC7
S123EEBE8678BDEE1C7EEED6FE1C2CEE00BDEDF2FE1C2C0808FF1C2C33323962737200696E
S123EEDE6C6C6567616C206F70636F6465003B000203040512131415181C1D1E1F1A21386D
S123EEFE3A3C3D4142454B4B4E5152555B5E6162656B7172757B83878F939DA3B3C3C7CC05
S123EF1ECDCFD3DCDDE3ECEDF3FCFD006E6F7000000000007461700074706100696E7800D9
S123EF3E64657800636C760073657600636C630073656300636C69007365690073626100BF
S123EF5E6362610000000000746162007462610000646161000061626100000000006272DD
S123EF7E61000062686900626C73006263630062637300626E650062657100627663006230
S123EF9E76730062706C00626D690062676500626C740062677400626C6500747378006948
S123EFBE6E730070756C610070756C620064657300747873007073686100707368620000F5
S123EFDE727473000072746900000077616900737769006E6567000000636F6D006C737209
S123EFFE0000726F72006173720061736C00726F6C006465630000696E6300747374006A9E
S123F01E6D7000636C72007375626100636D706100736263610000616E6461006269746197
S123F03E006C646161007374616100656F72610061646361006F72616100616464610063B3
S123F05E7078006A7372006C647300737473007375626200636D7062007362636200006171
S123F07E6E64620062697462006C646162007374616200656F72620061646362006F7261E8
S114F09E6200616464620000006C64780073747800C9
S123F0AF3637B61D86272A4AFF1D84F61D851BB71D854FB91D84B71D84FE1D84F61D865A9D
S123F0CF6D002604095A26F8A60009BDF2B95A2AF733323936B61D866F00084A26FA3239FA
S123F0EF3637F61D864FAA002604085A26F83332393637B61D86FE1D88E60008FF1D88FEBD
S123F10F1D8AE70008FF1D8A4A26EB3332393637B61D86FE1D880C6900084A26FA333239B9
S123F12F3637B61D88F61D893637FB1D868900B71D88F71D89F61D86FE1D880C6600085ABB
S123F14F26FA3332B71D88F71D893332393637B61D860CFE1D88E600FE1D8AE20008FF1D7A
S123F16F8AFE1D88E70008FF1D884A26E63332393637B61D860CFE1D88E600FE1D8AE900DF
S123F18F08FF1D8AFE1D88E70008FF1D884A26E6333239363733323936860836304F562486
S123F1AF02AB0168016A0026F5313139FF1D8DCEF1F67F1D8CE001A20025057C1D8C20F598
S123F1CFEB01A90036FF1D8FFE1D8DB61D8C8B30A7003208FF1D8DFE1D8F08088CF20026FC
S123F1EFD1FE1D8D6F0039271003E80064000A00013637FF1D6DF61D6D4FCE1D65BDF1BBCC
S123F20FCE1D65BDF22D862EBDF24EF61D6E4FCE1D65BDF1BBCE1D68BDF37D33323936A67B
S122F22F002603092007813026030820F2BDF37D32394D61746820696E636C75646564E5
S123F24E36413239B6C008850227F932B7C009395139B6C0084424FAB6C0093936B660003C
S123F26E848026F932B7400039B66000840127F9B64000393637CE1C09C6048DECA70008BB
S123F28E5A26F8FE1C0B33323936860D8DB2860A8DAE3239CEF7FCBDF37D3936FF1C11B6A4
S123F2AE1C118D07B61C128D0232393636444444448D098D8B328D048D863239840F810A14
S123F2CE2D038B37398B30393637CE1C365FBDF25E810D2606A7006F012037810A27F681B3
S123F2EE1127EB811327E781082704817F26165D27DC8608BDF24E8620BDF24E8608BDF27C
S123F30E4E095A20C9C15027C5BDF24EA700085C20BCCE1C36FF1C3433323937CE0000FF4F
S123F32E1C11FE1C3486206D00273FA100260608FF1C3420F2A60027318120272D810D27E9
S123F34E29810A272508803081112D028007840FFF1C34CE1C11C6040C690169000C5A2689
S123F36EF7AA01A701FE1C3420CBFE1C1133397D1D5D26FB3686FFB71D5DA600270608BDC5
S123F38EF24E20F6087F1D5D32398D0986144A26FDB6C012393637F6C010C4C78407484862
S123F3AE481BB7C01033323937F61D58C480270737C609F71D5F334D2704C47F2002CA80CC
S123F3CEF71D58333937F61D584D2704CA082002C4F7F71D58333937F61D584D2704CA04BA
S123F3EE2002C4FBF71D58333937F61D58C4FC84031BB71D583339CE1C3639FE1CA0A600ED
S123F40EE6013936374D260DB6C0138A08B7C01384F7B7C013333239364D2607B61D5B8423
S123F42E7F2005B61D5B8A80BDF50D32393637F6C0101784C78AB8B7C010863C4A26FDB671
S123F44EC0128D72F7C0103332393637F6C0101784C78A88B7C010863C4A26FDB6C0128DF2
S123F46E23F7C0103332393637F6C0101784C78AB0B7C010863C4A26FDB6C0128D06F7C09B
S123F48E1033323936CE0000FF1D6380212A014F48B71D63FE1D6332393637F6C0101784D8
S123F4AEC78AA8B7C010863C4A26FDB6C0128D06F7C0103332393637CEF4E916C40F5D2786
S123F4CE0508085A20F8EE00FF1D6144444444BB1D61B71D61FE1D61333239060006060678
S123F4EE0C06120619061F0625062B06320638063E0644064B06510657065D070007067D39
S123F50E1D5C26FB37C6FFF71D5CB71D5B3686083630F6C010C4FCF7C01068012402CA02D2
S123F52EF7C010CA01F7C0106A0026E9C4FCF7C0103131337F1D5C3937C6FED700812823FC
S123F54E030D2035F6C010C4FBF7C010CE00C8BDE3A8B11D5F2722F61D5F5CC129270A5F4C
S123F56E5C7C00007D00002710F71D5FF6C010CA04CE00C8BDE3A820CB33393637840F4869
S123F58E4848BDF50D4FBDF4113332395FB61D58848026015C174D2603C60939F61D5F390A
S123F5AE3637B61D6FF61D70B71D73F71D74B61D71F61D72B71D75F71D76CE1D73333239A0
S123F5CECE1D7A39FF1D80CE1D7AFF1D82FE1D8086FFE600C1992261C40FC109225BE600F9
S123F5EEFE1D82E700FE1D80E601C159224BC40FC1092245E601FE1D82E701FE1D80E60279
S123F60EC1592235C40FC109222FE602FE1D82E702FE1D80E603C123221FC40FC10922198A
S123F62EE603FE1D82E703FE1D80E6045D270AC1072206FE1D82E7044F39B71D7739B61DDE
S109F64E7739013901398E
S123F654BDF27781052EF9B71C08B61C08260ABDF282BDF277A70020E78101260ABDF282F2
S123F674A600BDF26A20D981022607BDF282AD0020CE81032609BDF2824FBDF26A20C18190
S123F694042609BDF2824FBDF26A20B4810526B04FBDF26ABDF26A8668BDF26A8602BDF297
S106F6B46A209D28
S123F6B7B6C0101684C78AF8B7C010BDF738B6C01281472213BDF738B6C01281472209CE99
S123F6D7F767BDF37D7EF7011784C78AC8B7C010BDF738B6C0128148233BBDF738B6C012C4
S123F6F781452331CEF783BDF37DCEF740BDF37DBDF2978602BDF648CE03E8BDE3A88601DD
S123F717BDF6484FBDF3B6B61D5B8478BDF50D4FBDF41120E3F7C010CE0DACBDE3A87EF617
S123F737B736863C4A26FD32390D0A53797374656D20706F776572696E6720646F776E2008
S123F757696E203130207365636F6E64730D0A000D0A4261747465727920766F6C74616771
S123F7776520746F6F206C6F770D0A000D0A4865617473696E6B2074656D706572617475C9
S111F797726520746F6F20686967680D0A0040
S123F7A50D0A2020202020202020202045415253206D61696E20636F6E736F6C65206D6FEA
S123F7C56E69746F7220202856312E32290D0A20202020202020202020202020202020392C
S123F7E5202D204665627275617279202D20313939310D0A0D0A001B5B481B5B4A00556EA3
S123F8056B6E6F776E20636F6D6D616E640D0A0046756E6374696F6E206E6F7420696E737B
S123F82574616C6C6564207965740D0A004E6F206A756D70206164647265737320676976BB
S123F845656E0D0A00557365722070726F6772616D2072657475726E656420736166656C4A
S123F865790D0A00466C616773203D20000D0A426164206C6F61642E20436865636B737593
S123F8856D206572726F722E000D0A4C6F7765737420616464726573732077726974746520
S123F8A56E2020746F2069732024000D0A4869676865737420616464726573732077726913
S123F8C57474656E20746F2069732024005374617274656420726F6F742070726F636573BA
S123F8E5730D0A0053746172746564207061725F7365632070726F636573730D0A004B69B7
S123F9056C6C6564206C6173742070726F63657373207375636365737366756C6C790D0AEE
S123F9250050726F636573732320204F776E6572232020537461636B2020202050430D0AEE
S123F9450050726F63657373207461626C652066756C6C2C2063616E6E6F7420737461721B
S123F96574206A6F620D0A0050726F6365737320494420756E6B6E6F776E0D0A004E6F20E8
S123F98570726F6365737320494420676976656E0D0A0053746172746564206C6F77207089
S123F9A5726F636573730D0A0046756E6374696F6E2063616C6C206E6F7420696E636C75EA
S123F9C5646564005374617274656420737461745F636F6D2070726F636573730D0A000D5D
S123F9E50A4261747465727920766F6C7461676520697320000D0A4865617473696E6B207D
S123FA0574656D706572617475726520697320000D0A416972207465726D70657261747577
S123FA25726520697320000D0A4E5652414D20766F6C74616765206D656173757265732078
S123FA45002D002D00480049004E005A004F76004300710068656C70003F0063006400657D
S123FA6500720067006C0075007073007374617274006B696C6C00656E7600726164696FAE
S123FA856E00726164696F666600636F6D706F66660000E769E7E5E7E5E7ECE85EE912EA44
S123FAA5ECEAB2EBF2EA15E9BDE9C5E9EAE5A2ED02ED0CED1571202E2E2E2E2E2E2E2E2E12
S123FAC52E2E2E2E2E2E2E2051756974206D6F6E69746F722070726F6772616D0D0A3F2062
S123FAE52E2E2E2E2E2E2E2E2E2E2E2E2E2E2E2E205072696E742068656C7020696E666F5B
S123FB05726D6174696F6E0D0A63203C73746172743E203C656E643E202E2E20436C6561BE
S123FB257273206D656D6F727920616464726573732072616E676520746F202430300D0A2D
S123FB4564203C73746172743E203C656E643E202E2E2044756D7020626C6F636B206F664D
S123FB65206D656D6F72790D0A65203C73746172743E202E2E2E2E2E2E2E2E204564697449
S123FB852F76696577206D656D6F72792E204279746520617420612074696D650D0A6720F4
S123FBA561646472657373202E2E2E2E2E2E2E2E20426567696E20657865637574696F6ECD
S123FBC5206F662070726F6772616D0D0A72202E2E2E2E2E2E2E2E2E2E2E2E2E2E2E2E2066
S123FBE55072696E74207265676973746572206C6973740D0A6C202E2E2E2E2E2E2E2E2E4D
S123FC052E2E2E2E2E2E2E204C6F616420646174612066726F6D20636F6E736F6C652069CF
S123FC256E20686578207265636F726420666F726D0D0A75203C73746172743E203C656EF2
S123FC45643E202E2E20446973617373656D626C65722070726F6772616D206F70636F6432
S123FC6565730D0A7073202E2E2E2E2E2E2E2E2E2E2E2E2E2E2E205072696E742062616364
S123FC856B67726F756E642070726F63657373207461626C650D0A656E76202E2E2E2E2EB4
S123FCA52E2E2E2E2E2E2E2E2E205072696E742073656E736F7220646174610D0A726164AE
S123FCC5696F6E202E2E2E2E2E2E2E2E2E2E2E20537769746368206F6E20746865207261D8
S123FCE564696F0D0A726164696F6666202E2E2E2E2E2E2E2E2E2E20537769746368206FC0
S123FD0566662074686520726164696F0D0A636F6D706F6666202E2E2E2E2E2E2E2E2E2E91
S123FD25205475726E206F66662074686520636F6D70757465720D0A73746172742061647C
S123FD456472657373202E2E2E2E20426567696E206261636B67726F756E642070726F6388
S123FD6565737320617420616464726573730D0A6B696C6C2070726F6365737323202E2EB3
S123FD852E2E205465726D696E617465206261636B67726F756E642070726F636573730DC9
S123FDA50A0A203C73746172743E206D65616E73207374617274206164647265737320694D
S123FDC573206F7074696F6E616C20616E64203C656E643E20697320616C736F206F7074BF
S10EFDE5696F6E616C0D0A200D0A00AE
S10BFFF8E3BEE4B7E40AE000F3
S9030000FC
